:020000020000FC
:1000000026C0189503C01CC01895189506B2032287
:1000100004FC0126102C1F1813FC0FC014FE1895A9
:10002000F02C27BB222705E003BF0BE802BF02E04C
:1000300008BF09BF00E205BF189522E014FC24E0C8
:10004000B998BA9800E305BFE3BEE9BE1895EE245F
:10005000222738E118E038BBC09AF6B2F322F4FC4C
:10006000F12600E20BBF00E305BF78948895FECF30
:10007000686166746D616E6E23736F66747761720A
:02008000650019
:00000001FF
